:100000000C944E050C94AF050C9492080C94AF051B
:100010000C94AF050C94AF050C94AF050C94AF0590
:100020000C94AF050C94AF050C940D160C94AF0511
:100030000C94D3230C94AF050C94AF050C94AF052E
:100040000C94AF050C94AF050C94AF050C94AF0560
:100050000C94AF050C9428240C94AF050C94AF05B8
:100060000C94AF050C94AF050C94AF050C94AF0540
:100070000C94AF050C94AF050C94AF050C94AF0530
:100080000C94AF050C94AF050C94AF050C94AF0520
:100090000C94AF050C94AF050C94AF050C94AF0510
:1000A0000C94AF050C94AF050C94AF05620A640A7A
:1000B000700A700A700A700A700A700A660A680A82
:1000C0006A0A700A700A640A720A700A700A2C0AB4
:1000D000620A700A700A680A700A700A700A700A66
:1000E000700A700A6A0A620A4E0A700A520A700A94
:1000F000700A700A2E0A660A700A700A5C0A700A90
:10010000700A700A300A6E0A700A500A700A640A8D
:10011000700A700A600A540A700A560A680A700A5D
:10012000700A700A5E0A580A700A700A700A700A29
:10013000700A700A700A5A0A700A320A700A700A43
:10014000660A700A700A6E0A700A700A700A700AEB
:10015000700A700A700A700A700A340A700A700A0B
:10016000700A5C0A700A700A700A700A700A700AD3
:10017000700A700A700A700A360A700A380A3A0A57
:10018000700A700A700A3C0A3E0A400A700A420A63
:10019000440A700A700A700A6C0A460A700A4A0A0F
:1001A000480A4C0A700A700A700A700A6E0A960AA7
:1001B000A40AB00AB00A880AB00AB00AB00AB00AA3
:1001C000B00AB00AB00AB00AB00AB00AB00AB00A5F
:1001D000B00A8A0AB00A8C0AB00AB00AB00AB00A99
:1001E000A80AB00ABF0AA60AB00AB00AB00AB00A42
:1001F000B00AB00AB00AB00AB00AB00AB00AB00A2F
:10020000B00A800A9C0A8E0AA00AB00A900AB00AB4
:10021000940AB00A9E0A920AA20A980A9A0AB00A96
:10022000B00AB00AB00AB00AB00AB00A820A840A58
:10023000860AAA0AAC0AB00AB00AB00AAE0A8E0B45
:10024000AC0BB80BDC0BEC0BF80B140C2B0C4E0CA2
:100250006B0CF60C220D9B0DCD0DB70DDE0DF00DC8
:10026000F80DFE0D020E080E640E660E680E6A0E84
:10027000AA0E720E720E720E6C0E6E0E700E5B1463
:1002800082147A1582147A15CE14F1147A15481551
:100290005715D319D3190B1A0B1A861A9A1C9A1CC4
:1002A0009A1CBA1A9A1C621A621A541C9A1C691C6B
:1002B000871C007B46010203763A687F6577482BEE
:1002C000353B6978796439141E3C6A7A1D16041A24
:1002D0001F3D6B061B070821203E6C2C19091715C2
:1002E000223F6D11050B0A1C23406E7E100D182451
:1002F00025416F360E0C122726427037380F331304
:100300002D43717534322F2E44727C7D2830317428
:10031000457351504A524D492A5466594F5C5F4CBF
:100320004B4E62635A5D5E60295367585B56576156
:1003300047554842403E3C3A3B456843413F3D2B90
:10034000357E697A790078141E7C6A7B1D16041A42
:100350001F7F6B061B070821204D6C2C19091715F0
:10036000224A6D11050B0A1C234C6E49100D1824EE
:1003700025516F360E0C1227264F7037380F331366
:100380002D52717534502F2E4E72397D28306531C3
:100390004B735464586776012A773259745C5F66F0
:1003A000020362635A5D5E60295344575B56556190
:1003B000474680291E1F20212223242526272D2E53
:1003C0002A2B141A0815171C180C12132F30287812
:1003D000041607090A0B0D0E0F33343579311D1B36
:1003E00006190511103637387D557A2C393A3B3CC1
:1003F0003D3E3F4041424353475F6061565C5D5E16
:1004000057595A5B62634648324445677B7F6503B0
:1004100001025250514F68696A6B6C6D6E6F70715A
:10042000725800494C754A4D734B4E767C777E74FA
:10043000665472253032582000623A2530345820F4
:1004400000652530325820002146554C4C212000B3
:100450002146462120007725303258200021435381
:10046000335F4630210A00214353335F52454144F4
:1004700059210A00214353325F45305F4630210A3B
:1004800000214353325F4630210A00214353325F3B
:100490004530210A00214353325F494E4954210A15
:1004A00000214353315F45305F25303258210A0027
:1004B0000A5B4F56525D20004C2575200053257570
:1004C00020000A49443A2530345828256429200060
:1004D0004D6F7573653A206E6F7420737570706F11
:1004E000727465640A005225752000572575200036
:1004F0005725752000572575200058257520004187
:100500002575200049257520005B4348475D200084
:100510000A5052543A25303258204953523A253025
:10052000345820005B5253545D20000A4552523A21
:1005300025303258204953523A2530345820000A89
:100540004B6579626F6172642073746172742E0AF4
:10055000000A55534220636F6E6669677572656461
:100560002E0A000A0A544D4B3A3662373164383845
:10057000312F4C5546410A0A003403490042004DD0
:100580000020005000430020006B006500790062ED
:10059000006F00610072006400200063006F006E55
:1005A0000076006500720074006500720000000EA5
:1005B0000374002E006D002E006B002E000000045E
:1005C00003090409027400040100A03209040000B8
:1005D000010301010009211101000122400007056A
:1005E000810308000A090401000103000000092139
:1005F000110100012236000705820308000A0904E0
:100600000200020300000009211101000122220062
:1006100007058303200001070503032000010904E7
:10062000030001030000000921110100012239002B
:10063000070584032000011201100100000008EDED
:10064000FEEE1B01000102000105010906A10105E2
:100650000719E029E71500250195087501810205B4
:1006600008190129059505750191029501750391F8
:10067000010507190029F71500250195F875018175
:1006800002C00631FF0974A1010975150026FF009B
:100690009520750881020976150026FF00952075C2
:1006A000089102C005010980A101850216010026FA
:1006B00037001A81002AB700751095018100C00526
:1006C0000C0901A1018503160100269C021A0100F4
:1006D0002A9C02751095018100C005010906A1013F
:1006E000050719E029E71500250195087501810224
:1006F0009501750881010508190129059505750100
:1007000091029501750391010507190029FF150054
:1007100026FF00950675088100C0636F6E73756DC6
:1007200065723A20253034580A0073797374656D08
:100730003A20253034580A000A002530325820006B
:100740006B6579626F6172643A20004C45443A20CF
:10075000253032580A0025583A2530386225730A68
:10076000000A202030313233343536370A006465D0
:100770006C5F6B65795F6269743A2063616E2774A0
:100780002064656C3A20253032580A006164645F49
:100790006B65795F6269743A2063616E27742061CA
:1007A00064643A20253032580A003F00433E20005E
:1007B0004C25640A000A092D20436F6E736F6C6527
:1007C000202D0A4553432F713A09717569740A0047
:1007D0000A092D204D61676963202D0A643A096476
:1007E000656275670A783A096465627567206D61AC
:1007F000747269780A6B3A096465627567206B6583
:1008000079626F6172640A6D3A0964656275672086
:100810006D6F7573650A763A0976657273696F6EE6
:100820000A733A097374617475730A633A09636FE2
:100830006E736F6C65206D6F64650A302D343A09F4
:100840006C61796572302D34284631302D4634295B
:100850000A506175733A09626F6F746C6F616465F9
:10086000720A6E3A094E4B524F0A003F004E4B52ED
:100870004F3A206F66660A004E4B524F3A206F6E19
:100880000A0074696D65725F72656164333228298C
:100890003A202530346C580A006B6579626F6172BA
:1008A000645F6E6B726F3A2025580A006B6579623F
:1008B0006F6172645F69646C653A2025580A006B49
:1008C0006579626F6172645F70726F746F636F6C71
:1008D0003A2025580A00686F73745F6B6579626F00
:1008E0006172645F6C65647328293A2025580A0098
:1008F0000A092D20537461747573202D0A00474333
:10090000433A20352E342E30204156522D4C494248
:10091000433A20322E302E30204156525F4152430E
:10092000483A20617672350A004F5054494F4E5371
:100930003A204C5546412045585452414B45592088
:10094000434F4E534F4C4520434F4D4D414E442055
:100950004E4B524F204B45594D41505F53454354E8
:10096000494F4E20424F4F544C4F414445525F53E4
:10097000495A450A004255494C443A2036623731BB
:1009800064383831202830343A32373A3236204E03
:100990006F762032322032303230290A00564944F4
:1009A0003A2030784645454428742E6D2E6B2E290A
:1009B000205049443A203078316265652849424DDB
:1009C000205043206B6579626F61726420636F6EA3
:1009D00076657274657229205645523A2030783017
:1009E0003030310A00444553433A20636F6E7665D8
:1009F00072742049424D205043206B6579626F61CB
:100A0000726420746F205553420A000A092D205643
:100A1000657273696F6E202D0A000A6D6F757365BC
:100A20003A206F66660A000A6D6F7573653A206F2B
:100A30006E0A000A6B6579626F6172643A206F66B4
:100A4000660A000A6B6579626F6172643A206F6EA4
:100A50000A000A6D61747269783A206F66660A004E
:100A60000A6D61747269783A206F6E0A000A6465D3
:100A70006275673A206F6E0A000A64656275673AAC
:100A8000206F66660A000A0A626F6F746C6F616499
:100A900065722E2E2E2000433E20000011241FBE22
:100AA000CFEFDAE0DEBFCDBF04B603FE41C08091D8
:100AB000880390918903A0918A03B0918B038730BA
:100AC000904BA740B04BA1F5109288031092890378
:100AD00010928A0310928B0314BE0FB6F894A89557
:100AE00080916000886180936000109260000FBE6A
:100AF0001092010810920008E3E0F0E089E0809392
:100B00005700E491E695E370E150E33040F4F0E003
:100B1000EE0FFF1FE35DFE4F8081918102C080E0F8
:100B200090E1E0E0F0E8E81BF90BF695E795099510
:100B300011E0A0E0B1E0EAE5FCE402C005900D920E
:100B4000A433B107D9F723E0A4E3B1E001C01D92BB
:100B5000A838B207E1F70E9470110C942B260C9470
:100B60000000FF93EF93E0913401F091350130974D
:100B700009F00995EF91FF910895FC01859180306E
:100B800011F0EFDFFBCF0895FF27E0E230E247FFEF
:100B90000CC0419597FF09C0EDE260957095809576
:100BA0009095611D711D811D911D27FF02C021952A
:100BB00030E350E2AA27660F771F881F991FAA1FEC
:100BC000A41710F0A41B63955A95A9F7AA3008F052
:100BD000A95FA05DAF93F39561157105810591053E
:100BE00041F7ED3211F4EF93F395F21718F43F93B8
:100BF000F395FBCF8F91B5DFFA95E1F70895E99171
:100C0000F9918591803021F0853219F0AADFF9CF72
:100C1000089520E0E89455915532C1F3503311F412
:100C2000689455915A3348F4505390F3220F022E92
:100C3000220F220F200D250FF4CF0EF4219589915C
:100C40009991533619F3533729F1533559F1BC01B2
:100C500088279927E8945C3621F4899199916894C2
:100C60005591543639F446EF7EF077FF0DC08FEF83
:100C70009FEF0AC055374AE039F0583540E121F07E
:100C8000523642E009F00895FF93EF937DDFEF9134
:100C9000FF91B7CFFF93EF93FC0181918030B9F3BF
:100CA00060DFFBCFFF93EF9368DFF1CFDF93CF934C
:100CB000CDB7DEB72596A3DFCF91DF910895282F1A
:100CC00080914101823071F08330B1F0813001F5C3
:100CD000E62FF0E038E0739FE00DF11D1124EE5493
:100CE000FC4F13C0E62FF0E088E0789FE00DF11D87
:100CF0001124EE5CFC4F09C0E62FF0E038E0739F52
:100D0000E00DF11D1124EE54FD4FE491E03819F48B
:100D100080E090E008959E2F9077892F90E034E056
:100D2000959587953A95E1F738E0239F800D911DC1
:100D3000112444E0880F991F4A95E1F7EF709C0158
:100D40002E0F311DF901EE0FFF1FE050F84985917C
:100D5000949108955998519A08955198599A0895DF
:100D60005898509A08955098589A08955198599AB9
:100D700085E08A95F1F7000089B186958170089524
:100D80005098589A85E08A95F1F7000089B18170F2
:100D90000895CF93DF93EC010E94B606882341F0BB
:100DA000209731F085E08A95F1F700002197F4CF84
:100DB000CE01DF91CF910895CF93DF93C2E3D0E0CE
:100DC0000E94B606811108C0209731F085E08A950F
:100DD000F1F700002197F4CFCE01DF91CF91089574
:100DE0002E9826982F9827980E94AA060E94B3064C
:100DF000E9E6F0E0808188608083E9980895E19ACF
:100E0000E99A0E94AD060C94B306E9980E94AA06DE
:100E10000C94B306CF93DF932FB7F894C0910201DF
:100E2000D0910301CE01882781159F4F19F080E0F2
:100E30009FEF02C08FEF90E08C2B9D2B90930301CE
:100E4000809302012FBFCE0199278F3F910581F535
:100E5000CD2FDD27C03FD10551F0CF3FD10509F49B
:100E600051C080917503C034D10599F407C08091B9
:100E7000750380FF33C080E594E004C080FF2EC07E
:100E800088E494E09F938F930E9456060F900F90F2
:100E900025C080FF37C0DF93CF9381E494E09F9318
:100EA0008F930E9456060F900F900F900F902AC0BC
:100EB000CE018F6F019699F08091750380FF0CC071
:100EC000DF93CF9389E394E09F938F930E9456061C
:100ED0000F900F900F900F90CD2F01C0CFEF80910A
:100EE000750380FF0CC01F92CF9382E394E09F9321
:100EF0008F930E9456060F900F900F900F908C2F9B
:100F000090E002C08FEF9FEFDF91CF910895CF93D4
:100F1000CAE1C15069F00E940A078F3F2FEF920784
:100F200049F48FE99FE00197F1F700C00000F1CF8D
:100F30008FEF9FEFCF91089510923A0110923901EF
:100F4000109238011092370180E090E890930101EF
:100F5000809300018FEF9FEF909303018093020134
:100F60000895EF92FF920F931F93CF93DF93082F73
:100F7000109237018091750380FF0CC01F920F9370
:100F800086E594E09F938F930E9456060F900F90F2
:100F90000F900F90E9980E94AA060E94B3068FE86E
:100FA00091E00197F1F700C000000E94B0068FE8C1
:100FB00091E00197F1F700C000000E94AD0680E1CA
:100FC00097E20E94C906892B11F481E07FC0C0E03E
:100FD000D0E0FF24F39410E0EE24E39490E59A959A
:100FE000F1F7C8010C2E02C0959587950A94E2F797
:100FF00080FF04C0FE240E94B30602C00E94B00617
:101000000E94DC06892B11F482E060C082E390E04C
:101010000E94C906892B11F483E058C02196C8307C
:10102000D105E1F680E58A95F1F7FF2019F00E94DD
:10103000B30602C00E94B0060E94DC06892B11F4A0
:1010400084E044C082E390E00E94C906892B11F439
:1010500085E03CC090E59A95F1F70E94B3060E94A6
:10106000DC06892B11F486E031C082E390E00E9417
:10107000C906892B19F0C2E3D0E009C087E026C079
:10108000209759F025E02A95F1F7000021970E945A
:10109000C0068111F5CFCD2B11F488E017C00E9456
:1010A000DC06892B19F0C2E3D0E009C089E00EC04C
:1010B000209759F085E08A95F1F7000021970E946A
:1010C000C0068823A9F3CD2BB9F48AE080933701B9
:1010D000809137018061809337010E94AD060E94A4
:1010E000B306E19AE99A8FEF9FEFDF91CF911F91BD
:1010F0000F91FF90EF9008958FEF9FEF9093030172
:10110000809302010E949C070E94AD060E94B306D4
:10111000E19AE99ADF91CF911F910F91FF90EF90A3
:101120000C9487071F920F920FB60F9211242F93E2
:101130003F934F935F938F939F9329B18091760351
:1011400040910001509101014115504819F48093DC
:1011500036010FC090913601891B833050F0809189
:1011600000019091010190933A018093390180E24E
:10117000DDC0809100019091010196958795909333
:1011800001018093000120FF09C08091000190912E
:10119000010190689093010180930001809100010A
:1011A0009091010199278038910509F4F9C0A8F4BC
:1011B0008032910509F4F4C038F4009709F4F0C0C6
:1011C000409709F489C0A9C08034910509F4E8C0AA
:1011D0008035910509F480C0A0C0803C910539F1AB
:1011E00050F48039910509F477C0803A910509F0EF
:1011F00094C084E64DC0803D910509F46DC0803EE9
:10120000910509F08AC080910001909101019093AD
:101210003A01809339018091000190910101892F59
:101220009927909301018093000183E252C084E6E4
:1012300049990FC0882369F095E09A95F1F700006D
:101240008150F6CF882349F095E09A95F1F7000098
:1012500081504999F7CF8111A3C0809100019091ED
:10126000010190933A01809339018091000190919E
:101270000101892F9927909301018093000182E257
:1012800028C0882379F095E09A95F1F70000815005
:10129000499BF7CF07C0882349F095E09A95F1F76D
:1012A000000081504999F7CF81117AC080910001E7
:1012B0009091010190933A0180933901809100014E
:1012C00090910101892F992790930101809300014A
:1012D00081E28093380133C0809100019091010137
:1012E00090933A018093390180910001909101011E
:1012F00097FF02C080E101C081E1809338018091B5
:1013000000019091010146E0969587954A95E1F795
:10131000909301018093000112C08091000190918F
:10132000010190933A018093390180E8809337015D
:101330008091370190E0982F88278F6F27C0809188
:1013400000019091010199278F3F910511F480EFE1
:10135000EDCF809103018F3F31F0809102018F3FEB
:1013600011F080E4E3CF8091020190910301982F66
:10137000882790930301809302012091000130910E
:1013800001018091020190910301822B909303014E
:101390008093020180E090E8909301018093000126
:1013A0009F918F915F914F913F912F910F900FBE21
:1013B0000F901F901895CF93C82F8DEE0E94B10704
:1013C0008A3F910521F48C2FCF910C94B107CF91D6
:1013D0000895E82FE695E695E695EF70F0E0EB5B73
:1013E000FE4F4081282F277081E090E002C0880FD7
:1013F000991F2A95E2F7242F30E028233923232B45
:1014000011F4842B80830895E82FE695E695E69500
:10141000EF70F0E0EB5BFE4F2081382F377081E0FA
:1014200090E002C0880F991F3A95E2F7422F50E0F2
:1014300048235923452B19F08095822380830895F2
:10144000482F50E0FA013397E138F10508F048C021
:10145000EA5AFF4F0C94252687E108958FE10895FD
:101460008CE5089580E6089582E6089587E2089560
:1014700083E508958FE2089589E3089587E3089549
:101480008FE3089587E408958FE4089586E508952D
:101490008EE508958FE7089580E0089585E6089524
:1014A0008EE608958FE6089580E3089588E3089511
:1014B00080E4089588E4089580E5089587E5089517
:1014C0008FE5089588E1089588E0089580E2089501
:1014D00080E1089589E108958DE6089588E20895F0
:1014E0008F7708958FE00895CF93482F50E0FA0149
:1014F0007C97E834F105A0F5E952FF4F0C942526BE
:1015000085E53EC08AE53CC08BE53AC08CE538C035
:101510008DE536C08EE534C08FE532C080E630C040
:1015200081E62EC082E62CC083E62AC08FE628C062
:1015300081E726C082E724C084E722C085E720C077
:1015400087E71EC088E71CC08AE71AC08CE718C06E
:101550008FE716C080E714C089E712C08BE710C080
:10156000C82F1F928F9381EA94E09F938F930E94DC
:1015700056060F900F900F900F908C2F01C084E5AE
:10158000CF9108950F931F93CF93DF930E9401246F
:101590008C010E940A07EC01019631F4C8010E94F7
:1015A0001924843F9140A8F3CE01DF91CF911F9180
:1015B0000F9108950E94F0060C94FF068091750328
:1015C000816080937503E5E4F1E0119281E0E535F7
:1015D000F807D9F70895E82FF0E0EB5BFE4F808124
:1015E0000895E5E4F1E0119281E0E535F807D9F7D7
:1015F0000895982F80914101823048F092FB88270E
:1016000080F990FD826091FD84600C94DB0908955F
:10161000CF93DF9380913701882371F18091390155
:1016200090913A01209137019F938F931F922F93AE
:101630008BE295E09F938F930E945606809137012D
:1016400080750F900F900F900F900F900F9071F486
:10165000809140018B3051F484E295E09F938F9309
:101660000E945606109240010F900F901092370181
:1016700010923A011092390180913801882309F4BF
:1016800040C090913801809144019817D1F1809128
:10169000390190913A01209138019F938F931F92C5
:1016A0002F9380E195E09F938F930E94560680913F
:1016B00044010F900F900F900F900F900F9085FFA7
:1016C00004C09091380194FD06C084FF12C080913F
:1016D000380185FF0EC0809140018B3051F489E0C4
:1016E00095E09F938F930E945606109240010F90B1
:1016F0000F90809138018093440110923A0110922A
:101700003901E09140018E2F90E08C30910508F076
:1017100025C3FC01E15EFE4F0C9425260E940507BF
:101720000E9401249F938F9384E095E09F938F9371
:101730000E945606109241011092430110924201FC
:101740000E94F10A0E9483190E94012490933F0194
:1017500080933E0181E065C080913E0190913F0100
:101760000E941924893E934008F4F8C282E031C0F7
:101770000E949C070E94FF068FE99FE00197F1F706
:1017800000C000008FEF0E94B1078A3F910511F45D
:1017900086E001C083E0809340010E9401249F9372
:1017A0008F938FEF94E09F938F930E9456060F9034
:1017B0000F900F900F90D2C20E9405072E98269A84
:1017C0002F98279A0E94012490933F0180933E0115
:1017D00084E080934001C2C280913E0190913F011C
:1017E0000E941924853F914008F4B8C285E0F1CFEA
:1017F0002E9826982F9827980E949C070E94FF06F3
:101800000E9401249F938F938AEF94E09F938F937C
:101810000E9456060E94012490933F0180933E014E
:1018200086E080934001C3CF0E940A07019609F425
:1018300095C20E9401249F938F9385EF94E09F931C
:101840008F930E9456060E94012490933F0180933B
:101850003E0187E0E6CF80913E0190913F010E94DA
:101860001924853F914018F089E0809340010E943F
:101870000A07019609F472C20E9401249F938F9374
:1018800080EF94E09F938F930E9456060E9401245C
:1018900090933F0180933E0188E0C3CF80913E0149
:1018A00090913F010E941924853F914018F089E0F2
:1018B000809340010E940A07019609F44FC20E94DA
:1018C00001249F938F938BEE94E09F938F930E94BC
:1018D000560689E0A6CF82EF0E94B1078F3F2FEF17
:1018E000920789F08A3F910589F40E94C20A8F3FCE
:1018F0003FEF930771F0D82FCC270E94C20A9E01B8
:10190000282BC90108C08FEF9FEF05C08EEF9FEF16
:1019100002C080E090E090934301809342010E94D6
:1019200001249F938F9386EE94E09F938F930E9460
:10193000560680914201909143010F900F900F90B5
:101940000F90009711F482E02BC08F3F3FEF930779
:1019500011F481E025C08E3F2FEF9207A1F38F3F56
:10196000910559F480ED94E09F938F930E94560661
:10197000109241010F900F901FC09C0125583B4AC7
:101980002230310580F480EF0E94B1078A3F910533
:10199000D1F683E00E94B1078A3F9105A1F683E06A
:1019A0008093410109C0803B3FEB9307C1F3882737
:1019B00081159F4BA1F3C7CF809141011F928F9357
:1019C000809143018F93809142018F9382EC94E048
:1019D0009F938F930E9456068AE0809340010F9058
:1019E0000F900F900F900F900F90B8C10E9401249C
:1019F0009F938F938DEB94E09F938F930E94560655
:101A00000F900F900F900F9080914101823029F03C
:101A1000833039F488EF0E94B1070E94FB160E94C0
:101A2000F90A8BE0809340010E9401249F938F93D9
:101A300088EB94E09F938F930E9456060F900F902F
:101A40000F900F900E940A079C012F3F9FEF3907CC
:101A500009F484C12115310519F02F3F310569F4CE
:101A60000E94F10A0E94831980EB94E09F938F9368
:101A70000E9456060F900F9071C1909141019230D3
:101A800009F44CC0933009F4CBC0913009F066C121
:101A900090913D01923099F028F4992341F09130D2
:101AA000C1F039C0933061F1943081F134C0803E8F
:101AB00021F0813E51F482E005C081E003C08D3108
:101AC000D9F483E080933D0149C187FFE3C08F775C
:101AD0000DC1863301F118F48A3229F41CC08A3A08
:101AE000D1F0863BC1F087FD03C00E94740A0BC091
:101AF0008F770E94740A0DC08D3969F484E0E2CFBB
:101B0000853449F485E50E94E90905C0853C19F44E
:101B100085E50E94040A10923D0120C1E0913C013C
:101B20004E2F50E04930510508F077C0FA01E55DCD
:101B3000FE4F0C942526803E69F030F4833871F016
:101B4000843871F48FE757C0813E31F0803F41F413
:101B500081E05BC082E059C084E057C082E04BC0A6
:101B600087FF98C00E94F10A85E994E098C0893502
:101B700009F453C0803F19F0823119F44EC083E05C
:101B800044C010923C0187FD03C00E94200A82C01D
:101B90000E94F10A8BE894E082C0833821F08438F7
:101BA00021F48FE738C082E036C010923C0187FFF5
:101BB0009DC00E94F10A81E894E071C010923C013E
:101BC000823109F4CBC0893509F4C8C087FD03C050
:101BD0000E94200A8BC00E94F10A84E794E05FC053
:101BE000843121F0803FC9F486E00FC085E00DC04C
:101BF000873799F480E00E94E9090FC0843169F4C5
:101C000087E003C0803F49F488E080933C01A6C090
:101C1000873719F480E00E94040A10923C019EC0AC
:101C200090913B01913009F443C038F0923009F4AF
:101C300063C0933009F47FC091C0863809F168F41D
:101C40008338D1F020F4803819F582E06CC08438F4
:101C5000A9F08538E9F48BE01DC08C38A9F030F488
:101C6000873881F08B38A1F481E014C08D3871F091
:101C7000803F71F481E057C082E00CC08FE70AC05A
:101C800086E008C080E006C089E004C08AE002C0A7
:101C900087FD03C00E94E90961C087E694E09F9335
:101CA0008F930E9456060F900F901092400156C0DD
:101CB000482F50E0FA01E358F109EB30F10590F4B8
:101CC000EC5CFE4F0C94252682E045C08FE743C0B4
:101CD0008BE041C086E03FC081E03DC089E03BC071
:101CE0008AE039C010923B0187FD03C00E94040ABC
:101CF00035C08DE594E0D3CF853279F030F486316C
:101D000071F08E3199F480E00BC0863221F0803F73
:101D100069F483E008C08DE503C083E501C081E577
:101D20000E94E90905C080933B0118C00E94F10A96
:101D300010923B0113C08E3169F020F48631B1F767
:101D400081E509C0853221F0863281F78DE503C037
:101D500083E501C080E00E94040AEACF81E0DF91C0
:101D6000CF9108958091790208950895CF93DF93DC
:101D700000D01F92CDB7DEB720917F03243021F52C
:101D800023E029839B838A8382E08093E9008FEF9D
:101D90009091E800815095FD06C095ED9A95F1F778
:101DA00000008111F5CF8091E80085FF0DC040E073
:101DB00050E063E070E0CE0101960E94261380910E
:101DC000E8008E778093E8000F900F900F90DF91DE
:101DD000CF910895CF93DF9300D01F92CDB7DEB798
:101DE00020917F03243029F522E02983805891092E
:101DF0009B838A832093E9008FEF9091E8008150C4
:101E000095FD06C095ED9A95F1F700008111F5CF8B
:101E10008091E80085FF0DC040E050E063E070E095
:101E2000CE0101960E9426138091E8008E77809360
:101E3000E8000F900F900F90DF91CF910895CF930E
:101E4000DF93EC0190917F03943009F048C08091BA
:101E500014018823D9F0809115018823B9F090935B
:101E6000E90081E8815049F09091E80095FD05C0B6
:101E70009AE29A95F1F700C0F5CF8091E80085FFCE
:101E80002EC040E050E060E270E019C081E0809335
:101E9000E90081E8815059F09091E80095FD07C074
:101EA000EFE3F1E03197F1F700C00000F3CF80914C
:101EB000E80085FF14C040E050E068E070E0CE012B
:101EC0000E9426138091E8008E778093E80080E2DC
:101ED000FE01A9E5B2E001900D928A95E1F7DF914C
:101EE000CF910895CF93C0915701C1110BC00E94AB
:101EF0000D24643C79408105910520F081E08093B8
:101F00005701C1E08C2FCF910895FF920F931F933B
:101F1000CF93DF93D82F0FB607FE83C080917F0346
:101F2000843081F08091070190E0019620910901B1
:101F300030E0822393232091080130E08217930739
:101F400009F0CDC00E94720F811110C0809107016D
:101F500090E001962091090130E0822393232091A3
:101F6000080130E08217930709F0B9C00E940124EC
:101F70008C01C091E900CF709091EC00892F8170A5
:101F800090FD80E8C82B83E08093E90085E0F82E7F
:101F90008091EB0085FD42C08091EB0080FF3EC048
:101FA0008091EE0087FF3AC080910801909107016F
:101FB000981709F457C09091E80095FF8EC0E09102
:101FC0000501F0910601E80FF11D20818F5F9091CE
:101FD00009018923809308012093F1008091E80092
:101FE00085FDE2CF8091E80080FFDECF8091E800A0
:101FF0008E778093E800F0920401D6CF809107019C
:1020000090E001962091090130E0822393232091F2
:10201000080130E08217930709F44CC0CF70C093D9
:10202000E90040910701842F90E001962091090179
:1020300030E0822393232091080130E08217930738
:1020400009F450C0E0910501F0910601E40FF11D83
:10205000D083809107018F5F90910901892380933C
:10206000070140C08091E80085FF37C0D093F100A0
:1020700021E03091F3008091F20090E0932B892BC6
:1020800091F08091E80080FF0EC08091E80085FF0C
:1020900003C01092F100F9CF8091E8008E77809311
:1020A000E800F0920401222309F4A8CFCF70C09376
:1020B000E90018C080910401882309F4AFCF0E9481
:1020C00001249C018017910711F4890161CF90913F
:1020D0000401915090930401F8CF20E0CACF4091C1
:1020E0000701B0CF80E0DF91CF911F910F91FF905A
:1020F000089580917E03811104C00E9492150C9472
:10210000EF15089510927E030895089542E061EC62
:1021100081E00E949F1242E061EC82E00E949F12E7
:1021200042E261EC83E00E949F1242E261EC84E0B3
:102130000C949F1280918103833009F455C030F4D0
:10214000813071F0823009F48EC008958A3009F42C
:102150007AC08B3009F460C0893009F09CC020C07F
:1021600080918003813A09F096C08091E800877FD2
:102170008093E8008091840390918503892B21F45A
:1021800060E289E592E003C060E080E090E070E00A
:102190000E9473138091E8008B778093E800089584
:1021A00080918003813209F076C080918403909100
:1021B0008503009719F0039709F06DC08091E8003E
:1021C000877F8093E8008091E80082FD05C08091C0
:1021D0007F038111F8CF5FC08091F1008093790275
:1021E0008091E8008B7753C080918003813A09F099
:1021F00052C08091840390918503892B09F04BC0D4
:102200008091E800877F8093E8008091E80080FF5C
:10221000FCCF8091140136C0809180038132D9F5C2
:102220008091840390918503892BA9F58091E80022
:10223000877F8093E8000E94D4128091820380936C
:1022400014010C94831980918003813221F58091CF
:10225000E800877F8093E8000E94D4128091830376
:1022600080937A02089580918003813AA1F480914D
:10227000E800877F8093E8008091E80080FFFCCF32
:1022800080917A028093F1008091E8008E778093AC
:10229000E8000C94D412089580917902809358013B
:1022A000109279020E94F10A0C9483190C944C113B
:1022B0000E94AE2380917D03882329F00E94BB23D6
:1022C00081110C94891208950E94CF2380915801A6
:1022D0008093790208950C94641108950C946D1103
:1022E000CF9384B7877F84BF0FB6F894A895809169
:1022F0006000886180936000109260000FBE90E0E3
:1023000080E80FB6F89480936100909361000FBE4F
:1023100085E89FE00E9481238AE091E00E94F61602
:1023200083E695E00E94BD050E94DA0A0E94AA1782
:102330000E9492150E94EF1578940E94AC1780912C
:102340007F03843029F00E94DB160E946D11F7CFC5
:1023500081E595E00E94BD050E946E118FE395E036
:102360000E94BD05C3E080917F03853019F40E946F
:102370005811F9CF0E94B0172091E4003091E50088
:1023800080915501909156012817390709F468C0CA
:102390008091E4009091E50090935601809355015F
:1023A0000E94720F882309F45BC080917F03843000
:1023B00009F056C08091E9008F702091EC00922FB7
:1023C000917020FD90E8892BC093E9009091EB007B
:1023D00090FF43C09091EE0097FF3FC0909108019D
:1023E00020910701291709F12091E80025FF1DC060
:1023F000E0910501F0910601E90FF11D30819F5F29
:10240000209109019223909308013093F10090915B
:10241000E80095FDE3CF9091E80090FFDFCF909129
:10242000E8009E779093E800D9CF9091F300209137
:10243000F20030E0392B232B81F09091E80090FFDF
:102440000CC09091E80095FF03C01092F100F9CF05
:102450009091E8009E779093E8008F708093E90058
:102460000E94DB1680CF292F332723303105C9F096
:1024700060F42130310581F02230310509F041C08E
:1024800084E790E023EC35E040C021323105E1F0F3
:102490002232310531F135C082E190E027E336E0A8
:1024A00034C099278130910549F028F0029749F509
:1024B000E9E7F5E005C0EFEBF5E002C0EFEAF5E093
:1024C000849190E09F0121C064307105D0F4660FC3
:1024D000771FFB01EC5DFE4F2081318189E090E0A8
:1024E00014C06430710568F4FB01EE0FFF1FE45E59
:1024F000FE4F20813181FB01E85EFE4F808190E03C
:1025000004C080E090E020E030E0FA0131832083D5
:10251000089580E189BD82E189BD09B400FEFDCF47
:102520008091D8008F7D8093D8008091E0008260F8
:102530008093E0008091E00081FDFCCF0895982F0A
:10254000973068F59093E900981739F07091EC0096
:102550002091ED005091F00003C0242F762F50E021
:1025600021FD02C09F5FECCF3091EB003E7F3093A6
:10257000EB003091ED003D7F3093ED003091EB00AA
:1025800031603093EB007093EC002093ED0050939A
:10259000F0002091EE0027FDE5CF80E008958F70D8
:1025A0008093E90081E008958091800387FF11C046
:1025B0008091E80082FD05C080917F038111F8CFF2
:1025C00011C08091E8008B770BC080917F03882336
:1025D00049F08091E80080FFF8CF8091E8008E7785
:1025E0008093E80008952091E4003091E50095E69D
:1025F0004091EC00842F817040FF23C08091E8005F
:1026000080FD1DC080917F03882399F0853099F06B
:102610008091EB0085FD11C04091E4005091E500F0
:102620002417350729F3915011F09A01E1CF84E086
:10263000089582E0089583E0089581E0089580E0A0
:1026400008954091E80042FFDDCF0895CF92DF92D8
:10265000EF92FF920F931F93CF93DF93EC018B01C7
:102660007A010E94F312811135C0E114F10439F0AE
:10267000F70180819181081B190BC80FD91FC12C4C
:10268000D12C0115110529F18091E80085FD18C0B4
:102690008091E8008E778093E8000E94DB16E114B9
:1026A000F10449F0F70180819181C80ED91ED182D1
:1026B000C08285E00FC00E94F312882311F30AC084
:1026C00089918093F10001501109FFEFCF1ADF0AC1
:1026D000D8CF80E0DF91CF911F910F91FF90EF90C5
:1026E000DF90CF90089520918603309187032617BD
:1026F000370748F06115710539F42091E8002E770D
:102700002093E80001C0B901FC0120E061157105CA
:1027100079F180917F038823F1F18530F1F1809187
:10272000E80083FD3CC08091E80082FD2EC08091CE
:10273000E80080FFEBCF2091F3008091F20090E061
:10274000922B6115710551F08830910538F4219173
:102750002093F100615071090196F3CF21E00897B1
:1027600009F020E08091E8008E778093E800CECFDA
:102770002111CFCF0AC080917F03882361F085307B
:1027800061F08091E80083FD0AC08091E80082FF3B
:10279000F2CF80E0089582E0089583E0089581E01B
:1027A000089520918603309187032617370748F054
:1027B0006115710539F42091E8002E772093E80027
:1027C00001C0B901FC0120E06115710591F1809112
:1027D0007F03882309F440C0853009F43FC080910D
:1027E000E80083FD3DC08091E80082FD2FC080910C
:1027F000E80080FFE9CF2091F3008091F20090E0A3
:10280000922B6115710559F08830910540F424919F
:102810002093F1003196615071090196F2CF21E0C9
:10282000089709F020E08091E8008E778093E80017
:10283000CBCF2111CCCF0AC080917F03882361F0D8
:10284000853061F08091E80083FD0AC08091E80046
:1028500082FFF2CF80E0089582E0089583E008953A
:1028600081E008951F93CF93DF93CDB7DEB7AA978A
:102870000FB6F894DEBF0FBECDBFE0E8F3E0809165
:10288000F100819323E0E838F207C9F70E949A101B
:102890008091E80083FF2EC1809180039091810395
:1028A000492F50E04A30510508F024C1FA01E15C9B
:1028B000FE4F0C942526803821F0823809F01AC189
:1028C00008C080917C0390917D03992389F08260F8
:1028D0000FC0809184038F70873008F00BC1809304
:1028E000E9008091EB0085FB882780F91092E900D0
:1028F0009091E800977F9093E8008093F100109208
:10290000F100D1C0282F2D7F09F0F4C0882319F0E1
:10291000823061F0EFC080918203813009F0EAC01B
:10292000933009F080E080937D032EC08091820374
:1029300081112AC0809184038F702FEF280F2630D9
:1029400008F0D8C08093E9002091EB0020FF1CC064
:10295000933021F48091EB00806214C09091EB00E1
:1029600090619093EB0021E030E0A90102C0440F98
:10297000551F8A95E2F74093EA001092EA00809191
:10298000EB0088608093EB001092E9008091E800F2
:10299000877F8093E8000E94D412ACC08111AAC046
:1029A000109182031F778091E3008078812B8093C0
:1029B000E3008091E800877F8093E8000E94D412B2
:1029C0008091E80080FFFCCF8091E30080688093D5
:1029D000E300111102C082E001C083E080937F0315
:1029E00089C08058823008F085C080918203909120
:1029F00083038C3D53E0950779F583E08A838AE26F
:102A000089834FB7F894DE01139620E03EE051E24F
:102A1000E32FF0E050935700E49120FF03C0E295CC
:102A2000EF703F5FEF708E2F90E0EA3010F0C796A6
:102A300001C0C0968D939D932F5F243149F74FBFFE
:102A40008091E800877F8093E8006AE270E0CE0121
:102A500001960E94731316C06091840370918503E0
:102A6000AE014F5F5F4F0E943312BC01892B09F406
:102A700041C09091E800977F9093E80089819A8106
:102A80000E94D1138091E8008B778093E80032C0D8
:102A9000803881F58091E800877F8093E8008091FD
:102AA0007B038093F1008091E8008E7772CF8111D3
:102AB00021C0809182039091830399270297D4F4D7
:102AC0008091E800877F8093E80080918203809363
:102AD0007B030E94D41280917B03811106C08091F8
:102AE000E30087FD02C081E001C084E080937F03A2
:102AF0000E9486108091E80083FF0AC08091E80060
:102B0000877F8093E8008091EB0080628093EB00E8
:102B1000AA960FB6F894DEBF0FBECDBFDF91CF915E
:102B20001F9108950E9400160E940816E0EEF0E042
:102B3000808181608083E8EDF0E080818F77808301
:102B400019BCA7EDB0E08C918E7F8C9380818F7E35
:102B5000808310927E0308950F931F93CF93DF938A
:102B60000E9400160E940816C8EDD0E088818F7779
:102B7000888388818068888388818F7D888319BC59
:102B800010927F0310927B0310927D0310927C03BE
:102B900000EE10E0F80180818B7F80838881816066
:102BA000888342E060E080E00E949F12E1EEF0E066
:102BB00080818E7F8083E2EEF0E08081816080837F
:102BC000808188608083F80180818E7F8083888106
:102BD00080618883DF91CF911F910F910895E8ED77
:102BE000F0E080818F7E8083E7EDF0E0808181607E
:102BF000808384E082BF81E080937E030C94AC15D7
:102C0000E8EDF0E080818E7F80831092E2000895ED
:102C10001092DA001092E10008951F920F920FB601
:102C20000F9211242F933F934F935F936F937F9352
:102C30008F939F93AF93BF93EF93FF938091E100A6
:102C400082FF0BC08091E20082FF07C08091E1000B
:102C50008B7F8093E1000E94DA168091DA0080FF7A
:102C60001FC08091D80080FF1BC08091DA008E7F4A
:102C70008093DA008091D90080FF0DC080E189BD8A
:102C800082E189BD09B400FEFDCF81E080937F031E
:102C90000E94791005C019BC10927F030E94821017
:102CA0008091E10080FF19C08091E20080FF15C093
:102CB0008091E2008E7F8093E2008091E20080614B
:102CC0008093E2008091D80080628093D80019BC84
:102CD00085E080937F030E9456118091E10084FF7C
:102CE00030C08091E20084FF2CC080E189BD82E188
:102CF00089BD09B400FEFDCF8091D8008F7D8093FF
:102D0000D8008091E1008F7E8093E1008091E20005
:102D10008F7E8093E2008091E20081608093E200E8
:102D200080917B03882311F084E007C08091E30049
:102D300087FD02C081E001C083E080937F030E9491
:102D40006B118091E10083FF24C08091E20083FF3A
:102D500020C08091E100877F8093E10082E0809332
:102D60007F0310927B038091E1008E7F8093E100CE
:102D70008091E2008E7F8093E2008091E20080618A
:102D80008093E20042E060E080E00E949F120E9497
:102D90008510FF91EF91BF91AF919F918F917F919E
:102DA0006F915F914F913F912F910F900FBE0F90B8
:102DB0001F9018950895CF9380917F038823A1F0E9
:102DC000C091E900CF709091EC00892F817090FD47
:102DD00080E8C82B1092E9008091E80083FD0E94F2
:102DE0003214CF70C093E900CF9108959093800280
:102DF00080937F020895E0917F02F09180023097E6
:102E000021F00190F081E02D099480E00895EF9287
:102E1000FF920F931F93CF93DF93E0917F02F09186
:102E200080023097B1F18C010280F381E02D099589
:102E30008091750382FF2DC080FF04C080E497E07D
:102E40000E94BD05E80110E28AE3E82E87E0F82E33
:102E50008091750380FF0BC088811F928F93FF9232
:102E6000EF920E9456060F900F900F900F90115006
:102E700021961111EDCF8091750380FF0AC088E380
:102E800097E0DF91CF911F910F91FF90EF900C94FD
:102E9000BD05DF91CF911F910F91FF90EF900895A5
:102EA000CF93DF9320917D0230917E02281739075E
:102EB00009F190937E0280937D02E0917F02F09170
:102EC00080023097B9F0EC010680F781E02D09957A
:102ED0008091750382FF0EC080FF0CC0DF93CF93FB
:102EE0008AE297E09F938F930E9456060F900F906F
:102EF0000F900F90DF91CF910895CF93DF932091A2
:102F00007B0230917C022817390709F190937C02EB
:102F100080937B02E0917F02F09180023097B9F0BC
:102F2000EC010084F185E02D09958091750382FF05
:102F30000EC080FF0CC0DF93CF938AE197E09F9390
:102F40008F930E9456060F900F900F900F90DF9175
:102F5000CF9108950C9453180E94F8230C94DE0A24
:102F6000BF92CF92DF92EF92FF920F931F93CF9376
:102F7000DF9300D000D01F92CDB7DEB70E94080BC0
:102F800002E812E0F12C8F2D0E94EB0AB82EF80116
:102F9000C080C82639F4F3940F5F1F4FF0E1FF1291
:102FA000F2CF30C08091750381FD0E945418D12C5E
:102FB000EE24E3948C2D8E21F9F0D982FA8291E0EF
:102FC0008B2D8E2109F490E09B830E940124816067
:102FD000782F9D838C8349815A816B818D810E94DA
:102FE0008A1849815A816B817C818D810E94992345
:102FF000F80180818E258083D394EE0CF8E0DF12F7
:10300000D9CFC9CF8FEF89838A831B820E94012485
:103010008160782F9D838C8349815A816B818D815A
:103020000E948A180E9498230E94FB1690918102A8
:10303000891741F10E94FB168093810290917503DC
:1030400092FF0EC090FF0CC01F928F938BE497E00D
:103050009F938F930E9456060F900F900F900F90A2
:10306000809181020F900F900F900F900F90DF9141
:10307000CF911F910F91FF90EF90DF90CF90BF9075
:103080000C94AA230F900F900F900F900F90DF9148
:10309000CF911F910F91FF90EF90DF90CF90BF9055
:1030A00008950C94F90A0895EF92FF920F931F93DD
:1030B000CF93DF9381E697E00E94BD05C0E0D0E0AA
:1030C0008CE2E82E81E0F82E06E517E08C2F0E94B6
:1030D000EB0A0E948623FF92EF921F928F93DF9359
:1030E000CF931F930F930E94560621968DB79EB7DC
:1030F00008960FB6F8949EBF0FBE8DBFC031D105A4
:1031000029F7DF91CF911F910F91FF90EF900895D4
:1031100008950895CF93DF93CDB7DEB72B970FB601
:10312000F894DEBF0FBECDBF942F4F83252F588755
:1031300069877A878B874A855B85452B31F02F3FDE
:1031400031F481E09F3F19F403C081E001C080E0C9
:1031500080FD07C04F81588569857A858B850E94DF
:103160009923DE01119686E0FD0111928A95E9F717
:1031700085E0FE01379601900D928A95E1F749812D
:103180005A816B817C818D819E810E94941F2B9638
:103190000FB6F894DEBF0FBECDBFDF91CF9108957B
:1031A000CF93882309F465C0C82F8CEF8C0F813A28
:1031B00020F080E58C0F8E3248F48C2F0E94D225AF
:1031C000811157C08C2F0E947C220CC080E28C0F92
:1031D000883058F4C77081E001C0880FCA95EAF7BB
:1031E0000E942123CF910C945B238BE58C0F8330BD
:1031F00078F4C53A29F0C63A31F083E890E005C08A
:1032000081E890E002C082E890E0CF910C945017E2
:1032100088E58C0F873168F5C83A89F0C93A91F092
:10322000CA3A99F0CB3AA1F0CC3AA9F0CD3AB1F034
:10323000CE3AB9F0CF3AC1F080E090E017C082EE0C
:1032400090E014C089EE90E011C08AEE90E00EC0CC
:1032500085EB90E00BC086EB90E008C083EB90E03C
:1032600005C084EB90E002C087EB90E0CF910C9416
:103270007D17CF910895882349F19CEF980F913ADB
:1032800020F090E5980F9E3218F40E94CC220DC0D9
:1032900090E2980F983058F4877091E001C0990F30
:1032A0008A95EAF7892F0E9427230C945B239BE5DC
:1032B000980F933020F480E090E00C945017885AD7
:1032C000873120F480E090E00C947D1708958823E6
:1032D00021F00E9421230C945B230895882321F080
:1032E0000E9427230C945B2308950E9441230E948F
:1032F00010230E945B2380E090E00E94501780E042
:1033000090E00C947D170E9431230C947519CF9294
:10331000DF92EF92FF920F931F93CF93DF9300D032
:1033200000D01F92CDB7DEB76C010E94AC23811193
:1033300001C385E0F601DE01119601900D928A9598
:10334000E1F7F60140815181238134812115310556
:1033500031F05F3F31F481E04F3F19F403C081E069
:1033600001C080E080FDE6C2F601F280E580E294D3
:103370008FE0E82249835A83FB82722F3D832C839E
:103380006F2D8D810E94F8218C010E94F7210E94EF
:10339000E720E12FE295EF708E2F90E0FC01E75BD4
:1033A000FE4F0C942526812F807F1F70882311F0FB
:1033B0001295107FFF20B9F0112329F0812F0E9470
:1033C00034230E945B23802F0F900F900F900F905B
:1033D0000F90DF91CF911F910F91FF90EF90DF90B1
:1033E000CF900C94D018802F0E943B19112309F420
:1033F000A1C2812F0E943A230F900F900F900F903F
:103400000F90DF91CF911F910F91FF90EF90DF9080
:10341000CF900C945B23812F807F1F70803211F03E
:103420001295107F002319F0013009F12BC0FF2005
:10343000A9F0EE2059F1F1E0812FEF1228C00F9092
:103440000F900F900F900F90DF91CF911F910F91E0
:10345000FF90EF90DF90CF900C944423EE2021F06A
:1034600021E0E21609F466C20E9447234DC0FF2006
:10347000E9F085E08E1508F45DC20E941E238123C9
:1034800029F042C0FF20F1F1E11015C0812F0F900B
:103490000F900F900F900F90DF91CF911F910F9190
:1034A000FF90EF90DF90CF900C94671994E09E15F9
:1034B00008F440C229C0F601858180FF13C08F70D7
:1034C0008583E4CF003F09F472C108F03EC180E477
:1034D000800F803208F442C1FF2009F4D3C1EE20EE
:1034E00009F483C1802F0E94D018093309F0C3C1A9
:1034F000FFEF21EE84E0F15020408040E1F700C072
:10350000000018C2E110C0C1812F42C1812F8695F1
:103510008695837019F08130B9F00CC2FF2019F044
:10352000C801937002C080E090E00F900F900F9060
:103530000F900F90DF91CF911F910F91FF90EF901F
:10354000DF90CF900C945017FF2019F0C8019370B2
:1035500002C080E090E00F900F900F900F900F90BE
:10356000DF91CF911F910F91FF90EF90DF90CF905F
:103570000C947D17812F837009F070C0F110DAC1AF
:10358000202F229526952770220F220F602F6F7013
:10359000862F90E0A0E0B0E06C017D01022E04C017
:1035A000CC0CDD1CEE1CFF1C0A94D2F704FF12C0E9
:1035B0008FE090E0A0E0B0E004C0880F991FAA1F40
:1035C000BB1F2A95D2F7BC01CD01609570958095FF
:1035D000909503C060E070E0CB01169516951370CE
:1035E0001230B1F040F56C297D298E299F291130C8
:1035F00031F10F900F900F900F900F90DF91CF91BE
:103600001F910F91FF90EF90DF90CF900C940C21C1
:103610006C297D298E299F290F900F900F900F9074
:103620000F90DF91CF911F910F91FF90EF90DF905E
:10363000CF900C9426210E940C21C701B6010F9057
:103640000F900F900F900F90DF91CF911F910F91DE
:10365000FF90EF90DF90CF900C94F220FF2019F0B4
:10366000812F817001C08695882309F463C1202FC2
:10367000229526952770220F220F602F6F70862FBC
:1036800090E0A0E0B0E06C017D01022E04C0CC0C03
:10369000DD1CEE1CFF1C0A94D2F704FF12C08FE061
:1036A00090E0A0E0B0E004C0880F991FAA1FBB1FE4
:1036B0002A95D2F7BC01CD016095709580959095C3
:1036C00003C060E070E0CB011695169513701230C0
:1036D000B1F040F56C297D298E299F29113031F1F7
:1036E0000F900F900F900F900F90DF91CF911F913F
:1036F0000F91FF90EF90DF90CF900C94D3216C2925
:103700007D298E299F290F900F900F900F900F9079
:10371000DF91CF911F910F91FF90EF90DF90CF90AD
:103720000C94E5210E94D321C701B6010F900F90A0
:103730000F900F900F90DF91CF911F910F91FF90FD
:10374000EF90DF90CF900C94C121023F09F45EC04E
:1037500008F449C0033F09F46CC0BECE902F9071AD
:10376000E92E812F8F71FF2051F00E945A21802F66
:10377000EE2019F08295807F8ACE8F7088CE0E94CD
:103780007B21802FEE2019F08295807F01C08F7001
:103790000F900F900F900F900F90DF91CF911F918E
:1037A0000F91FF90EF90DF90CF900C946E19FF2057
:1037B000A9F0E4E0EE1508F4BDC0812F8F710F90E1
:1037C0000F900F900F900F90DF91CF911F910F915D
:1037D000FF90EF90DF90CF900C94A021F5E0FE15C4
:1037E00008F4A8C0EACFFF2099F0812F8F710F90C5
:1037F0000F900F900F900F90DF91CF911F910F912D
:10380000FF90EF90DF90CF900C945A21FF2069F346
:10381000812F8F710F900F900F900F900F90DF916D
:10382000CF911F910F91FF90EF90DF90CF900C946C
:103830007B21FF2089F0812F8F710F900F900F90C7
:103840000F900F90DF91CF911F910F91FF90EF900C
:10385000DF90CF900C9445210F900F900F900F9018
:103860000F90DF91CF911F910F91FF90EF90DF901C
:10387000CF900C944021033509F43ACE073409F077
:1038800059C036CEEE2021F2802F0F900F900F906E
:103890000F900F90DF91CF911F910F91FF90EF90BC
:1038A000DF90CF900C943B19412F4F70602FC601D1
:1038B0000E946D240F900F900F900F900F90DF914A
:1038C000CF911F910F91FF90EF90DF90CF900C94CC
:1038D000422001112FC0FF2069F10E9483192FEFB0
:1038E00080E792E0215080409040E1F700C0000066
:1038F0000F900F900F900F900F90DF91CF911F912D
:103900000F91FF90EF90DF90CF900C944E24412FB9
:103910004F70602FC6010F900F900F900F900F9077
:10392000DF91CF911F910F91FF90EF90DF90CF909B
:103930000C9470240F900F900F900F900F90DF91C8
:10394000CF911F910F91FF90EF90DF90CF9008954E
:103950001F93CF93DF9300D000D01F92CDB7DEB777
:10396000942F4983252F5A836B837C838D834C81CD
:103970005D81452B31F02F3F31F481E09F3F19F4F9
:1039800003C081E001C080E0182F117080FD31C0BC
:1039900049815A816B817C818D810E94F821292F78
:1039A00022952F702C3030F42A30A0F4225022308F
:1039B00030F022C02C30C9F02F30B9F01DC0853A4C
:1039C00028F48430C0F4823028F415C090E2980FB7
:1039D000983088F0883E30F4803E68F48450813A14
:1039E00058F409C0803F41F406C093FB112710F939
:1039F00003C010E001C011E0812F0F900F900F90D5
:103A00000F900F90DF91CF911F910895CF93DF9387
:103A100000D000D01F92CDB7DEB70F900F900F905F
:103A20000F900F90DF91CF910895CF93DF9300D047
:103A300000D000D0CDB7DEB726960FB6F894DEBF23
:103A40000FBECDBFDF91CF9108951F93CF93DF932A
:103A5000C091920216E080919302C81799F0D0E0CD
:103A60001C9FF0011D9FF00D1124EC56FD4F40816D
:103A7000518162817381848195810E94151D2196F7
:103A8000C770E9CFDF91CF911F9108954091C40293
:103A90005091C5026091C6027091C7028091C80220
:103AA0009091C9020C94151D0F931F93CF93DF9330
:103AB0008091C90282958F7009F05DC08091C60225
:103AC000882309F458C0809192021091930260916A
:103AD000C4027091C502C091C702D091C80291E0A2
:103AE0006F3F09F090E0292F06E0811709F443C0E9
:103AF000209721F07F3F21F030E003C031E001C08A
:103B0000322F90E030FD34C0089FF001099FF00D86
:103B10001124DF01AC56BD4F11963C91119737131C
:103B200027C03C91361324C012963C911297311154
:103B30001FC013964D915C9114974C1B5D0B483C34
:103B40005105B0F48091C9028F7080618093C902E1
:103B5000E756FD4F80818F708061808384EC92E016
:103B60000E948719DF91CF911F910F910C94251D11
:103B700001968770BACFDF91CF911F910F91089571
:103B80009F92AF92BF92CF92DF92EF92FF920F93EC
:103B90001F93CF93DF93CDB7DEB761970FB6F8943D
:103BA000DEBF0FBECDBF8C0185E0F801DE011D96A2
:103BB00001900D928A95E1F7F80140815181F280E0
:103BC000C380D4809091C4026091C5022091C70245
:103BD0003091C8022115310531F06F3F31F481E099
:103BE0009F3F19F403C081E001C080E0F82FF1701D
:103BF0009F2E80FD52C184ECA82E82E0B82EE0906A
:103C0000C602F601E21BF30BEE2009F4E8C0809136
:103C1000C902E83CF10508F0A4C0282F207F09F074
:103C200053C0561313C0491311C0EF2CF1100EC02E
:103C30008F7080618093C9020E94461DC5010E9459
:103C400087198091C902F80185835BC1C114D10431
:103C500031F05F3F31F481E04F3F19F403C081E060
:103C600001C080E080FD03C081E08F2502C080E0BC
:103C700090E0F82FF170EF2E80FF1CC0809192022F
:103C80002091930236E0821709F418C190E0389F22
:103C9000F001399FF00D1124EC56FD4F6181561350
:103CA00006C06081461303C06281F61203C001960C
:103CB0008770E9CFEF2CFF2009F423C18091C9025E
:103CC00081608093C90262C0561306C0491304C0C4
:103CD000F11002C0F801A7C04D875E87FF867C2DDA
:103CE000D98AC88A6F2D89890E94A81C882399F1D6
:103CF000FF2089F12091C902822F82958F7090E078
:103D0000029774F08091C4029091C50298878F83C6
:103D10001986DB86CA862C87CE0107960E948719F2
:103D200086E0F801A4ECB2E001900D928A95E1F7EB
:103D30000E94541D0E94461D11C0561749F14D871F
:103D40005E87FF867C2DD98AC88A6F2D89890E945B
:103D5000A81C81112CC0C8010E948719EE24E3948D
:103D6000D0C0282F207F49F77C2DD98AC88A6F2D93
:103D700089890E94061D84EC92E00E94871986E0E2
:103D8000F50111928A95E9F70E94461DE12CB9C010
:103D90004913D5CFF110D3CFF8018583C8010E9414
:103DA000871986E0F50111928A95E9F7AAC0FF20EC
:103DB00091F22091C902822F82958F7090E0029734
:103DC0000CF4AECF8091C4029091C5029A8389838E
:103DD0001B82DD82CC822E83CE0101969FCFE83CF0
:103DE000F10508F04BC0EF2CFF2009F4B4CF5613B7
:103DF00030C049132EC02091C90220FD21C0822F5E
:103E000082958F70482F50E041155105C9F0F80197
:103E100025834F30510541F08F5F982F9295907F09
:103E2000822F8F70892B8583C8010E94871986E0B5
:103E3000F801A4ECB2E001900D928A95E1F72AC056
:103E400086E0F801A4ECB2E001900D928A95E1F7CA
:103E500058C04D875E87FF867C2DD98AC88A6F2D12
:103E600089890E94A81C81115BCF8091C902816061
:103E70008093C902C8010E94871943C07C2DD98A4A
:103E8000C88A6F2D89890E94061D86E0F50111926E
:103E90008A95E9F70E94461D34C0FF2009F45BCFE4
:103EA0004D875E87FF867C2DD98AC88A6F2D8989C8
:103EB0000E94A81C882309F44ECF32CF7C2DD98ACA
:103EC000C88A6F2D89890E94F821292F22952F7089
:103ED000223028F49F7039F0811105C00BC02430C6
:103EE00028F49F7049F4805E883020F0C8010E9459
:103EF00087199E2CE92C05C0F8019581907F99F7D0
:103F0000F9CF8E2D61960FB6F894DEBF0FBECDBFF0
:103F1000DF91CF911F910F91FF90EF90DF90CF90A5
:103F2000BF90AF909F9008951F93CF93DF93CDB72D
:103F3000DEB72C970FB6F894DEBF0FBECDBF4F8310
:103F4000588769877A878B879C87CE0107960E945E
:103F5000C01D8823D1F09F8188852A853B85232B2E
:103F600031F08F3F31F481E09F3F19F403C081E0CD
:103F700001C080E080FD47C04F81588569857A8502
:103F80008B859C850E94151D3EC086E0FE013796FC
:103F9000DE01119601900D928A95E1F7FF81E88587
:103FA0006A857B856115710531F0EF3F31F481E061
:103FB000FF3F19F403C081E001C080E080FD23C011
:103FC0002091930230E0C9010196877099274091B2
:103FD000920250E084179507F1F1F983EA837D831B
:103FE0006C8396E0929FD001939FB00D1124AC5644
:103FF000BD4FFE01319601900D929A95E1F78093A5
:1040000093020E94251D16E08091920290919302E6
:10401000891771F1189FC00111248C569D4F0E9481
:10402000C01D882329F1E09192021E9FF001112406
:10403000EC56FD4F4081518162817381848195816D
:104040000E94151D8091920290E001968770992739
:1040500080939202D9CF0E948319109293021092FA
:104060009202E4ECF2E086E0DF011D928A95E9F726
:104070002C960FB6F894DEBF0FBECDBFDF91CF9167
:104080001F910895DF92EF92FF920F931F93CF93AA
:10409000DF93FC01892B09F488C0E12CF12CDD248D
:1040A000D394EF0121968491853709F460C058F4C8
:1040B000843708F04EC0843008F068C08130D1F0F9
:1040C000823071F172C0883709F45BC050F48637D2
:1040D00009F453C0873709F068C08E2D0E942E2343
:1040E00052C09CE7980F903708F05FC08F770E940E
:1040F0003B194EC08F010E5F1F4FFE01849190E26D
:10410000980F983050F48770FD2D01C0FF0F8A95ED
:10411000EAF78F2F0E94342315C00E94D01814C0D4
:104120008F010E5F1F4FFE01849190E2980F98302F
:1041300068F48770FD2D01C0FF0F8A95EAF78F2F75
:104140000E943A230E945B23E80122C00E943B198F
:10415000FBCFCF010296FE01C491CC2361F0EFE9C1
:10416000FFE03197F1F700C00000C150F6CFCF015A
:104170000296FE01F490EC010BC00E941E23E82E73
:1041800007C00E9431230E945B2302C00E94D01806
:104190008F2D882341F0EFE9FFE03197F1F700C060
:1041A00000008150F6CFFE017CCFDF91CF911F91AF
:1041B0000F91FF90EF90DF90089560934A03709302
:1041C0004B0380934C0390934D030C94A9230895C3
:1041D00060934E0370934F03809350039093510369
:1041E0000C94A8230F931F9300914E0310914F033B
:1041F0002091500330915103602B712B822B932B14
:1042000060934E0370934F03809350039093510338
:104210001F910F910C94A8230F931F9300914E03AD
:1042200010914F032091500330915103602371236B
:104230008223932360934E0370934F038093500324
:10424000909351031F910F910C94A8230F931F93E8
:1042500000914E0310914F03209150033091510370
:10426000602771278227932760934E0370934F0333
:1042700080935003909351031F910F910C94A823A6
:1042800060E070E0CB010C94DD200F931F9341E0C0
:1042900050E060E070E08A019B0104C0000F111F34
:1042A000221F331F8A95D2F7C901B8011F910F91C0
:1042B0000C94DD200F931F9341E050E060E070E02C
:1042C00004C0440F551F661F771F8A95D2F780914F
:1042D0004A0390914B03A0914C03B0914D038A0186
:1042E0009B01082B192B2A2B3B2BC901B8011F91CD
:1042F0000F910C94DD200F931F9341E050E060E09C
:1043000070E004C0440F551F661F771F8A95D2F7CF
:10431000409550956095709580914A0390914B031C
:10432000A0914C03B0914D038A019B0108231923EE
:104330002A233B23C901B8011F910F910C94DD2062
:104340000F931F9341E050E060E070E004C0440F21
:10435000551F661F771F8A95D2F780914A03909167
:104360004B03A0914C03B0914D038A019B01082798
:1043700019272A273B27C901B8011F910F910C94D7
:10438000DD200F931F9300914A0310914B0320915E
:104390004C0330914D03602B712B822B932B1F917B
:1043A0000F910C94DD200F931F9300914A031091FD
:1043B0004B0320914C0330914D03602371238223E2
:1043C00093231F910F910C94DD200F931F93009165
:1043D0004A0310914B0320914C0330914D03602709
:1043E0007127822793271F910F910C94DD20089548
:1043F0008F929F92AF92BF92DF92EF92FF920F93B4
:104400001F93CF93DF9300D000D01F92CDB7DEB7BC
:104410006B837C838D838A018C819D81892B31F014
:104420001F3F31F481E04F3F19F403C081E001C028
:1044300080E080FF03C080E090E04DC08B81882346
:10444000D1F180904A0390904B03A0904C03B09020
:104450004D0380914E0390914F03A0915003B09172
:104460005103882A992AAA2ABB2A8FE1E82EF12C27
:10447000D501C4010E2C04C0B695A79597958795D4
:104480000A94D2F780FD06C081E0E81AF10880F7AF
:10449000D12C07C0DE2CB8018E2D0E945F0601973B
:1044A00099F388E0189FF0011124E653FD4FE00FC7
:1044B000F11DD08209C088E0189FF0011124E65355
:1044C000FD4FE00FF11DD08009831A8369817A8145
:1044D0008D2D0E945F060F900F900F900F900F9000
:1044E000DF91CF911F910F91FF90EF90DF90BF90E0
:1044F000AF909F908F90089590911401992379F136
:1045000090911501992359F1982F96959695969526
:104510009F31A1F0E0911601F0911701E90FF11D13
:10452000877021E030E0A90102C0440F551F8A9531
:10453000E2F7CA019181892B8183089590917503D7
:1045400090FF29C01F928F938CE897E09F938F93E1
:104550000E9456060F900F900F900F900895209193
:10456000160130911701F90132969FEF40E0519109
:10457000851789F09F3F19F4511101C0942F4F5FA7
:104580004E31A9F79F3F39F0F901E90FF11D97FD71
:10459000FA9582830895089590911401992381F1E9
:1045A00090911501992361F1982F9695969596957E
:1045B0009F31A9F0E0911601F0911701E90FF11D6B
:1045C000877021E030E0A90102C0440F551F8A9591
:1045D000E2F7CA01809591818923818308959091A2
:1045E000750390FF1CC01F928F938EE697E09F93F8
:1045F0008F930E9456060F900F900F900F90089582
:10460000E0911601F09117019F01225E3F4F9281C8
:10461000891301C012823196E217F307C1F708959A
:1046200081E090E0E0911601F0911701E80FF91F89
:104630001082019680329105A9F708958091740344
:10464000089590917403892B809374030895809545
:104650009091740389238093740308958093740365
:10466000089510927403089590917303892B809399
:104670007303089580959091730389238093730346
:104680000895109273030895809352030895109231
:10469000520308958091160190911701FC01319603
:1046A0009C01205E3F4F80E0919191118F5FE21756
:1046B000F307D1F70895E0911601F0911701809169
:1046C00074038083E0911601F0911701908180912D
:1046D0007303892B808380915203882361F0E091DA
:1046E0001601F09117019081892B80830E944A2343
:1046F00081111092520380911601909117010C9430
:104700000717909335018093340108958295982F6F
:10471000937344E0949F900111248C7C8695869538
:10472000282B822F8575880F2A7A2695822B08954B
:104730000895CF93DF9300D000D01F92CDB7DEB79E
:104740000F900F900F900F900F90DF91CF910895E1
:10475000089508950C94511880E0089583B7817FDF
:104760008C6083BF83B7816083BF7894889583B75B
:104770008E7F83BF0895CF930E9488180E94080BF4
:104780000E948918C0E08C2F0E94EB0A811104C09E
:10479000CF5FC031C1F701C081E0CF9108950E9481
:1047A000F10A0C9483191F920F920FB60F921124E5
:1047B0008F939F93AF93BF938091760390917703EC
:1047C000A0917803B09179034196A11DB11D80930A
:1047D000760390937703A0937803B0937903BF9106
:1047E000AF919F918F910F900FBE0F901F901895D2
:1047F00082E084BD93E095BD9AEF97BD80936E00F3
:1048000008952FB7F8948091760390917703A09143
:104810007803B09179032FBF08952FB7F894609172
:1048200076037091770380917803909179032FBF7D
:1048300008959C014FB7F894809176039091770387
:10484000A0917803B09179034FBF821B930B089519
:1048500078941F920F920FB60F9211248F939F930B
:10486000AF93BF938091760390917703A0917803E3
:10487000B09179030196A11DB11D809376039093A9
:104880007703A0937803B0937903BF91AF919F9181
:104890008F910F900FBE0F901F9018950E94921548
:1048A000F89487E797E7909301088093000887E0E2
:1048B00090EBDC018093880390938903A0938A0393
:1048C000B0938B039CE088E10FB6F894A895809391
:1048D00060000FBE90936000FFCF80E090E00895ED
:1048E0000895CF93C82F1F928F9380EB97E09F93EB
:1048F0008F930E94560681E090E0A0E0B0E0BC01FA
:10490000CD0104C0660F771F881F991FCA95D2F783
:104910000E94E8200F900F900F900F90CF910C9471
:104920008319CF938732A8F58E3108F02BC18031DF
:1049300009F49FC0F8F4873009F464C0A8F4863005
:1049400009F024C180917503817F8E7F8093750368
:1049500085EB97E00E94BD0587E99AE00E94BD05BE
:1049600081E080937A034CC08B30F1F18E3009F4F2
:104970006CC00CC1863109F4B0C020F4813109F457
:10498000EDC004C1893109F491C08B3109F449C0EB
:10499000FDC0883349F150F4893209F4F1C0853300
:1049A00009F4EEC0873209F0F1C0EAC0833409F49B
:1049B000E7C028F48A3308F4E9C08953E4C0883496
:1049C00009F0E4C00E94831986E89AE00E94BD05C0
:1049D0002FEF83ED90E3215080409040E1F700C03D
:1049E00000000E944E240CC080ED97E05CC08DE674
:1049F0009AE00E94BD0580917503816080937503E4
:104A0000C1E0C9C080917503C82FC17080FFEFCF8E
:104A100089E79AE00E94BD0580917503817F8E7FB2
:104A20003DC09091750391FBCC27C0F981E0C82768
:104A3000892FC0FB81F980937503CC2319F080E6A0
:104A40009AE027C082E59AE02EC09091750392FB10
:104A5000CC27C0F981E0C827892FC0FB82F9809359
:104A60007503CC2319F083E49AE013C083E39AE042
:104A70001AC09091750393FBCC27C0F981E0C82739
:104A8000892FC0FB83F980937503CC2351F087E213
:104A90009AE00E94BD058091750381608093750343
:104AA0007AC08AE19AE00E94BD05AACF8BE09AE025
:104AB0000E94BD0585EE99E00E94BD058DE999E053
:104AC0000E94BD0585E799E00E94BD0589E299E055
:104AD0000E94BD058EEF98E0E6CF80EF98E00E943F
:104AE000BD050E94FB161F928F9386ED98E09F9361
:104AF0008F930E945606809114011F928F938FEB23
:104B000098E09F938F930E94560680917A021F929D
:104B10008F938CEA98E09F938F930E945606809122
:104B200015011F928F9389E998E09F938F930E94BC
:104B300056060E940D249F938F937F936F9382E874
:104B400098E09F938F930E9456068DB79EB7469626
:104B50000FB6F8949EBF0FBE8DBF52CF0E9483192F
:104B6000C091150181E0C827C0931501CC2329F01D
:104B700088E798E00E94BD050EC08DE698E093CFCF
:104B800080E001C08D510E9471243ACF8BE698E0FD
:104B90000E94BD05C0E08C2FCF91089580E008955C
:104BA0000C94CE25CF93C82F80917A03882319F0D7
:104BB000813059F042C0E0911601F09117018081D7
:104BC000823261F08434D9F509C0E0911601F09188
:104BD00017018081823211F0843461F48C2F0E949D
:104BE000D025811104C08C2F0E94912424C081E023
:104BF00090E021C08C2F0E94CE2581111BC0C431B2
:104C000089F018F4CB3029F010C0C93259F0C833FC
:104C100061F485EB97E00E94BD058CEA97E00E9465
:104C2000BD0508C010927A030CC08AEA97E00E9482
:104C3000BD0507C081E0817006C010927A0380E054
:104C400002C080E0F8CFCF910895EE0FFF1F0590CE
:0A4C5000F491E02D0994F894FFCFD1
:104C5A000080FFFF0559010000FFB20E1F0FB50EBD
:104C6A00EA0EB60E0101530340362239DA06A406CB
:104C7A0082064906D505EE05070627060000080044
:044C8A000400020020
:106800008800EA44E944E244040005000600070069
:10681000080009000A000B000C000D000E000F001C
:1068200010001100120013001400150016001700CC
:10683000180019001A001B001C001D001E001F007C
:10684000200021002200230024002500260027002C
:10685000280029002A002B002C002D002E002F00DC
:10686000300031003200330034003500360037008C
:10687000380039003A003B003C003D003E003F003C
:1068800040004100420043004400450046004700EC
:10689000480049004A004B004C004D004E004F009C
:1068A000500051005200530054005500560057004C
:1068B000580059005A005B005C005D005E005F00FC
:1068C0006000610062006300640065A185006700EC
:1068D000680069006A006B006C006D006E006F005C
:1068E0007000710072007300890087008A008B00BD
:1068F000E000E100E200E300E400E500E600E7007C
:106900000100010001000100EA4401000100E2442D
:106910000100010001000100460001004A004B0097
:10692000010001004700480001000100E9440100A6
:106930000100010001000100010001003A003B00DC
:106940003C003D003E003F0040004100420043004B
:10695000010035004C0039000100440045005200A0
:1069600049000100010050004F0029004D004E0079
:1069700051000100010001000100010001000100BF
:1069800001000100010001000100010001000100FF
:1069900001000100010001000100010001004D00A3
:1069A0004A004E004B0001000100010001000100FF
:1069B00001000100010001000100010001000100CF
:1069C00001000100010001000100010001000100BF
:1069D00001000100010001000100010001000100AF
:1069E0000100010001000100490001000100010057
:1069F000010001000100010001000100010001008F
:00000001FF
